:0800000077CC76CCACCC74CCBB
:1018C00017C016C04CC014C00902120001010080EC
:1018D0003209040000000000000012011001FF00A6
:1018E0000008D01653070B0100000001040309048F
:1018F00011241FBECFE5D2E0CDBFDEBF00EB0F93BA
:1019000007E00F9310E0A0E6B0E0E4EFFFE102C0D3
:1019100005900D92A636B107D9F720E0A6E6B0E013
:1019200001C01D92A639B207E1F7E2C1A82FB92F75
:1019300080E090E041E050EA609530E009C02D91F0
:1019400082279795879510F084279527305EC8F3F6
:101950006F5FA8F30895EADF8D939D930895CF9369
:10196000CFB7CF93C0915F02C03B21F4C0915E021C
:10197000C73021F0CF91CFBFCF91A1CFCC27C39556
:10198000B39BE9F7B39B0BC0B39B09C0B39B07C0E4
:10199000B39B05C0B39B03C0B39B01C0D3C00F92E0
:1019A000DF93C0917900DD27C058DF4F012EB39B34
:1019B00003C0DF910F90E6CF2F930F931F934F93A8
:1019C0002FEF4F6F06B303FB20F95F933F9350E077
:1019D0003BE065C016B30126502953FDC89556B3A8
:1019E000012703FB25F92F7306B3B1F05027102709
:1019F00013FB26F906B22230F0F000C016B301271F
:101A000003FB27F90126502906B22430E8F54F7769
:101A1000206816B30000F6CF50274F7D206206B233
:101A2000102F000000C006B300265029102713FB1A
:101A300026F906B2E2CF4F7B06B3206400C0DACFAE
:101A400001265029187106B269F14E7F2160012FDD
:101A500016B328C0002650294D7F06B22260102FF1
:101A600029C0012650294B7F06B22460012F2DC0CA
:101A700016B301265029477F2860000006B22EC009
:101A80004F7E06B3206130C0422706B3499300263B
:101A90005029102706B24FEF13FB20F9297F16B308
:101AA00079F2187159F10126502906B2012703FB7A
:101AB00021F9237F06B371F2002650293150D0F06E
:101AC00006B2102713FB22F9277E16B351F2012626
:101AD0005029012703FB06B223F92F7C49F20000AD
:101AE00006B3102713FB24F90026502906B22F79DC
:101AF00039F270CF10E21ABF002717C03B50319562
:101B0000C31BD04010E21ABF0881033CF9F00B342C
:101B1000E9F0209177001981110F1213EDCF0936EA
:101B200051F10D3211F0013E39F700937E003F91E3
:101B30005F914F911F910F912F91DF910F90CAB735
:101B4000C5FD1DCFCF91CFBFCF91189520917E00BD
:101B5000222369F310917C00112321F5343022F106
:101B600030937C0020937800109179003BE0311B8A
:101B70003093790019C000917C0001309CF40AE593
:101B80003091600034FD11C000936000CCE6D0E0DD
:101B900010C0052710E000C021C0052710E0C8953F
:101BA00008BB14C03AE501C032ED032EC0E0D0E01E
:101BB00032E017B31861C39A08B317BB58E120E8A5
:101BC0004FEF20FF052708BB279517951C3F28F7E7
:101BD00000004552B0F720FF0527279508BB179551
:101BE0001C3FB8F629913A9561F7077E10917D0068
:101BF000110F08BBC250D04011F01093770010E2D3
:101C00001ABF086017B3177E402F477E54E05A95DD
:101C1000F1F708BB17BB48BB8ACFF8942FEFB0E8A9
:101C2000A0E44AE0B1BF000081EE9CE0B399FECF92
:101C3000B39BFECF0197B399FDCF97FF03C0BA1BAB
:101C4000819501C0BA0FA69529F4281710F031B775
:101C5000282FA1E0415031F731BF0000789408955A
:101C6000F894F201329785E080935700E8957894D4
:101C70000895F201309729F49093680080936700EB
:101C800007C0E430F10539F490936A00809369004D
:101C90008FE59CEC1FC02CEB421628E1520639F46C
:101CA00080916700909168008E559C4F13C02EEB79
:101CB000421628E1520639F48091690090916A0039
:101CC0008D559C4F07C02AEB421628E1520611F4AD
:101CD00081B790E02FB7F89431E00C0130935700B2
:101CE000E89511242F0182E0480E511C2FBF089562
:101CF00004B603FC06C0EDEBF8E1E491EF3F09F018
:101D000068C114BE88E181BD87E081BDBB9A88E8C7
:101D100093E1ECE9F1E03197F1F70197D1F7BB9846
:101D2000AC9A8BB780628BBF7894C598712C8CE984
:101D300091E00197F1F7A895312C60917C00162F66
:101D4000135017FDB2C080917900CCE0D0E0C81BE1
:101D5000D109C058DF4F6150CE01E8DD8E3F9F446E
:101D600009F0A1C0809178008D3209F085C018304B
:101D700009F099C083EC80936C008AE58093600041
:101D8000109266009881292F207689812223D1F034
:101D9000712C811108C082E690E090937B008093C3
:101DA0007A0024E05FC0813051F481E180935700D4
:101DB000E8954C805D8097FD50C02FEF4FC0382EC6
:101DC00020E050C09A8110927500811106C01092D7
:101DD000760085E790E022E03BC0853019F49093CF
:101DE0007D002CC0863009F58B81813019F48AED95
:101DF00098E104C0823041F488EC98E190937B0034
:101E000080937A0022E10DC0833051F4911108C013
:101E10008CEE98E190937B0080937A0024E001C0DF
:101E200020E080E4809366001DC0883059F089303E
:101E300019F490937F0002C08A3039F085E790E072
:101E400020E006C08FE790E002C085E790E021E047
:101E500090937B0080937A0005C02E8180E8809368
:101E6000660007C08F81811104C08E81821708F43B
:101E7000282F2093610017C08091660087FF13C050
:101E800080EC481688E1580620F0842D8F7339F0D5
:101E90000AC089919991EDDE125091F7F6CF95E045
:101EA000392E1092610010927C008091600084FFB6
:101EB00042C0809161008F3F09F43DC0182F8930E6
:101EC00008F018E0811B8093610080916C0098E815
:101ED000892780936C00112311F1E0917A00F09131
:101EE0007B008091660086FF0BC0ADE6B0E0849178
:101EF0008D9331968DE690E0810F8A13F8CF0BC059
:101F0000EF01ADE6B0E089918D93FE018DE690E0A2
:101F1000810F8A13F8CFF0937B00E0937A00612F52
:101F20008DE690E018DD1C5F1C3019F08FEF809378
:101F300061001093600084E196B3987131F4815090
:101F4000D9F710927D0010927700C1E08111C0E0B6
:101F500080916B008C1729F0C11101C05EDEC09327
:101F60006B00C30101963C018035934C11F484E071
:101F7000382E872D8D7011F0BD9801C0BD9A232D8C
:101F80003320E9F08AE390E20197F1F72230A9F4D7
:101F9000F894E0ECF8E1E054F10983E08093570015
:101FA000E8953097C1F7412C512CC8E08FEF9FEF97
:101FB00060DEC150D9F754DE02C02530E1F384E081
:101FC0003812B5CEEDEBF8E1E491EF3F09F4AFCE76
:101FD000BD98F894BB9A1BBE15BA10925F02EAEB4B
:101FE000F8E1E4918E2F81508E3F10F4E1BF0000A4
:041FF00065CCFFCFEE
:061FF4005AFF18BA400874
:04000003000018C021
:00000001FF
